:020000040800F2
:1000000000040120010200080302000803020008A6
:1000100003020008030200080302000803020008AC
:10002000030200080302000803020008352F00083D
:10003000030200080302000803020008030200088C
:10004000030200080302000803020008030200087C
:10005000030200080302000891310008BD310008C6
:10006000E931000815320008413200080302000897
:10007000030200080302000803020008030200084C
:10008000030200080302000803020008030200083C
:100090000302000803020008030200086D32000892
:1000A000030200080302000803020008030200081C
:1000B000B52F00080302000803020008030200082D
:1000C00003020008030200080302000803020008FC
:1000D00003020008030200080302000803020008EC
:1000E000D5320008030200080302000803020008DA
:1000F00003020008030200080302000803020008CC
:1001000003020008030200080302000803020008BB
:1001100003020008030200080302000803020008AB
:10012000030200080302000803020008030200089B
:10013000030200080302000803020008030200088B
:100140000302000803020008030200083526000825
:10015000030200080302000803020008030200086B
:10016000030200080302000803020008030200085B
:10017000030200080302000803020008030200084B
:10018000030200080302000803020008030200083B
:10019000030200080302000803020008030200082B
:1001A000030200080302000803020008030200081B
:1001B000030200080302000803020008030200080B
:1001C00003020008030200080302000803020008FB
:1001D00003020008030200080302000803020008EB
:1001E00003020008030200080302000803020008DB
:1001F00003020008030200080302000803020008CB
:1002000002E000F000F8FEE772B6394880F3088893
:10021000384880F3098838484EF60851CEF200017C
:10022000086040F20000CCF200004EF63471CEF2CD
:1002300000010860BFF34F8FBFF36F8F40F20000E3
:10024000C0F2F0004EF68851CEF200010860BFF314
:100250004F8FBFF36F8F4FF00000E1EE100A4EF6A4
:100260003C71CEF200010860062080F31488BFF3D1
:100270006F8F01F063FE02F0E5FD4FF055301F492E
:100280001B4A91423CBF41F8040BFAE71C49194A4A
:1002900091423CBF41F8040BFAE71A491A4A1B4B3A
:1002A0009A423EBF51F8040B42F8040BF8E70020D5
:1002B0001749184A91423CBF41F8040BFAE701F094
:1002C00081FE02F029FE144C144DAC4203DA54F8BE
:1002D000041B8847F9E700F03FF8114C114DAC4280
:1002E00003DA54F8041B8847F9E701F069BE0000FF
:1002F000000401200024012000000008000001206B
:1003000000040120F83600080024012050240120B8
:100310005024012048340120000200080002000897
:1003200000020008000200082DE9F04F2DED108AB0
:10033000C1F80CD0D0F80CD0BDEC108ABDE8F08F1D
:10034000002383F311882846A047002001F0AEFA6D
:1003500001F05AFA00DFFEE71B4B792270B51A70E4
:100360006FF07F0200245A720E225C709C70DC7069
:100370001C715C719C71DC711C729A72DC7201F0F0
:10038000ABFD064601F0D4FD054650B90F4B9E4229
:1003900017D001339E4241F2883412BF0546002433
:1003A0000125002001F09EFD0DB100F0B7F800F02E
:1003B00011FD00F009FC204600F052F900F0AEF803
:1003C000F9E70446EDE700BF50240120010007B023
:1003D00008B500F09BFBA0F120035842584108BD2E
:1003E00007B5054B02211B88ADF8043001A800F0C9
:1003F000DBFB03B05DF804FBD0330008064991F83D
:10040000243033B100230822086A81F8243000F038
:10041000FFBB0120704700BF702401202DE9F84F79
:10042000234C94F824300546884617468BBB2E464D
:10043000DFF87C90002F38D094F824A0BAF1000F98
:1004400005D12022FF214846266200F0B1FCCAF106
:100450000805BD4228BF3D465FFA85FBAD00414619
:100460002A4604EB8A0000F079FC94F82430A7EBCC
:100470000B079B445FFA8BFBBBF1080F2E44A8448B
:10048000FFB284F824B0D5D1FFF7B8FF0028D1D14E
:1004900008E0266A06EB8306B042C9D0FFF7AEFF3C
:1004A0000028C4D10020BDE8F88F0120BDE8F88FF6
:1004B0007024012010B572B6202383F3118862B630
:1004C0001248C3680BB101F079FA0023104A0F48B3
:1004D0004FF47A7101F036FA002383F311880D4C42
:1004E000236813B12368013B2360636813B1636819
:1004F000013B6360084B1B7833B9636823B9022062
:1005000000F022FC3223636010BD00BF5C24012098
:10051000B5040008A0290120982401202DE9F0410C
:10052000454B464953F8042F013201D1BDE8F08113
:100530008B42F7D1424C434B22689A427AD9424BC4
:100540009B6803F1006303F5C0339A4272D2002026
:1005500000F056FB3D4B0220187000F0EDFB3C4BC9
:100560001A6C00221A64196E1A66196E596C5A6454
:10057000596E5A66596E596941F08001596159693D
:1005800021F0800159615969196941F000511961DF
:10059000196921F0005119611B6972B62D492E4B62
:1005A0000B601D682468BFF34F8FBFF36F8F2B4B19
:1005B000C3F88420BFF34F8F5A6922F480325A6106
:1005C000BFF34F8FD3F88020C2F3C906C2F34E3277
:1005D0005201B70743F6E07E02EA0E08384631467C
:1005E000013948EA000CB1F1FF3FC3F874C200F1D1
:1005F0004040F5D1203A12F1200FEDD1BFF34F8FDB
:10060000BFF36F8FBFF34F8FBFF36F8F5A6922F421
:1006100000325A610022C3F85022BFF34F8FBFF35C
:100620006F8F72B6202383F3118862B6AD4685F3CF
:1006300008882047BDE8F081FC7F01081C80010884
:1006400004800108FF7F0108502401209824012024
:100650000038024008ED00E00080010800ED00E0F5
:100660002DE9F04FB64C97B020228246FF210EA80C
:10067000A56800F09DFBB34A1378A046B3B9B24811
:1006800001211170C36072B6202383F3118862B612
:10069000C3680BB101F092F90023AC4AAA484FF4A9
:1006A0007A7101F04FF9002383F31188DFF8BCB2AF
:1006B000BAF1000F01D0CBF800A0A54F00243C7088
:1006C000CBF804402646012000F036FBBAF1000FBB
:1006D00000F0E081DBF80030002B40F0DB8117B048
:1006E000BDE8F08F0220FFF773FE002840F0D081B4
:1006F000984B1B88ADF82430022109A800F054FA69
:10070000E1E74FF47A7000F001FA031E0193EFDB8A
:100710000220FFF75DFE81460028E9D0019B581EAC
:100720000428E5D8DFE800F0030C0F12150016A826
:10073000052340F8343D042100F036FA4C4650E0E1
:1007400004217F48F8E704218348F5E70421834822
:10075000F2E71C24204600F055FA043409900421E5
:1007600009A800F021FA2C2CF4D1E7E7002EBFD025
:10077000002CBDD00220FFF72BFE064610B9012445
:100780002646B5E7012000F03BFA0220387000F061
:10079000D3FA0024E3B21846019300F041FA8146EF
:1007A00048B1019B184600F04BFA01340028F1D102
:1007B00034466B4B9DE7012302203B7000F0B2FAF8
:1007C0004D46D8F808309D4206D2284600F01AFA65
:1007D0000130EDD10435F4E700253D70CBF804502D
:1007E000344600F0EDFAFFF7FBFD4EE1002E3FF43A
:1007F0007FAF002C3FF47CAF0220387000F09CFAF1
:10080000322000F083F9041EB9DB14F00306B6D1E0
:10081000D8F808202B199342B1D8B4F5807FAED810
:10082000DFF84091A6420CDA4FF47A7000F06EF9CE
:100830000390039B002BA2DB039B06F809300136D3
:10084000F0E7C820FFF7C4FD0646002897D01F2D0B
:1008500011D8C5F12009A14528BFA1460EAB25F04E
:1008600003004A463F49184400F078FA4A46FF21FF
:100870003C4800F09DFA4FEAA4095FFA89F2394931
:100880002846FFF7CBFD0446002891D005EB8905EB
:100890000646A6E70220FFF79BFD00283FF428AF9D
:1008A000FFF7ACFD00283FF423AF4FF0000AD1461C
:1008B000D8F808309A453CD2BAF11F0F1CD80E9BCD
:1008C000013319D02AF0030316AA134453F8203C2D
:1008D000099325494B68A3B1002209A8135C83EA58
:1008E0000903DBB2013251F82330042A83EA1929C3
:1008F000F4D10AF1040ADBE7504600F083F90990CD
:10090000E7E71A46082012F0010F4FEA52021FBF14
:1009100082F06D4282F4380282F4034282F02002B7
:100920000138F0D141F823200133B3F5807FE8D1BD
:10093000D2E716A8042140F8489D00F035F950E7A9
:10094000502401209C2501205C240120B5040008CE
:1009500098240120D2330008542401205824012077
:10096000D43300089C240120A0250120A0290120C7
:1009700016A8002340F8343D642100F0F1F8002867
:100980007FF4B6AE0220FFF723FD00283FF4B0AE9F
:10099000099800F067F916AB43F8440D0421184696
:1009A000CBE716A8002340F8343D642100F0D8F8C6
:1009B00000287FF49DAE0220FFF70AFD00283FF4D7
:1009C00097AE099800F05CF916AB43F8400DE5E7E7
:1009D0000220FFF7FDFC00283FF48AAE00F056F934
:1009E00016AB43F83C0DD9E70220FFF7F1FC0028D5
:1009F0003FF47EAE09A9142000F04EF9814616A8F6
:100A0000042140F8389D00F0CFF8494609A894E742
:100A10004FF47A70FFF7DCFC00283FF469AEFFF773
:100A2000EDFC00283FF4C5AE0E9B01330CD008222C
:100A30000EA90020FFF7F2FC00283FF4BAAE2022F6
:100A4000FF210EA800F0B4F9FFF7CAFC2E4800F011
:100A500035FF44E616A8002340F8343D642100F039
:100A60007FF800287FF444AE0220FFF7B1FC002895
:100A70003FF43EAEFFF7B4FC41F2883000F01EFFB9
:100A8000099800F0D1F900F09BF94FF0000A1AE63E
:100A90000646A6E6002000F039F80390039B002BE1
:100AA000FFF614AE012000F03DF9039B213B122B11
:100AB0003FF609AE01A252F823F000BFE506000898
:100AC000030700086D070008C7060008C7060008EE
:100AD000C7060008ED070008C706000895080008CB
:100AE00071090008A3090008D1090008C706000819
:100AF000E9090008C7060008110A0008E307000812
:100B0000C7060008550A0008A086010037B5114B3A
:100B10001A780132D2B20024012A01468DF807402A
:100B200011D80D4803681D6A4FF47A734B430122B4
:100B30000DF10701A847012805D1084B9DF80700D2
:100B40001C7003B030BD4FF4FA7000F0B7FE4FF0E8
:100B5000FF30F6E700240120F0290120AC29012014
:100B600038B50E4B1A780132D2B2012A05460ED89A
:100B70000B4803681C6A4FF47A734B4304222946DE
:100B8000A047042803D1074B0020187038BD4FF44C
:100B9000FA7000F093FE4FF0FF3038BD00240120C2
:100BA000F0290120AC29012030B4054C2368DD690F
:100BB000044B0A46AC460146204630BC604700BFA5
:100BC000F0290120A0860100F8B501F0B3F8094C26
:100BD000094E0A4F2070002530682378834207D9D8
:100BE00001F0A2F8336805440133BD423360F3D904
:100BF000F8BD00BFAD290120A8290120FF7F010019
:100C000001F056B900F1006000F5C030006870478F
:100C100000F10060920000F5C03001F0E1B8000082
:100C2000054B1A68054B1B789B1A834202D9104466
:100C300001F07AB800207047A8290120AD290120D1
:100C400038B5074D04462868204401F075F828B9E6
:100C500028682044BDE8384001F086B838BD00BFA0
:100C6000A829012010F0030308D1B0F5806F05D842
:100C700000F10050A0F57120006870470020704717
:100C8000014BC058704700BF20F4F01F014B18689B
:100C9000704700BF002004E0F0B5204B1E68204BD9
:100CA0001F885D6893F90840C6F30B02BA424FEA09
:100CB000164622D09F89BA4221D01F8BBA4206D154
:100CC00002220C2404FB02335D6893F90840B6F558
:100CD000805F16D041F201039E4208BF5A24421E93
:100CE0000A44013D0B46934215D215F9016F581C79
:100CF0004EB1034600F8016CF5E70022E1E701225E
:100D0000DFE74124EBE72C2582421D7001D9981CB6
:100D10005C70401AF0BD1846FBE700BF002004E0FD
:100D200004240120022802BF024B4FF480229A6162
:100D3000704700BF00000240022802BF014B04229E
:100D40009A61704700000240022801BF024A5369BD
:100D500083F00403536170470000024010B5002384
:100D6000934203D0CC5CC4540133F9E710BD0000BA
:100D700030B5441E14F9010F0B4660B193F90050D1
:100D8000854201F1010106D11AB993F90020801AB8
:100D900030BD013AEEE7002AF7D1104630BD000021
:100DA00002460346981A13F9011B0029FAD170472D
:100DB00002440346934202D003F8011BFAE770474E
:100DC000024B1A78024B1A70704700BFAC29012001
:100DD0000024012038B5104D104C284600F0A8F82A
:100DE0002146284600F0D0F823680D48DA6ED2F884
:100DF000043843F00203C2F8043800F05FFD0949EB
:100E0000206800F0D5F92368DA6ED2F8043823F0B0
:100E10000203C2F8043838BDF029012080340008EC
:100E200040420F00D03400087047000072B6202303
:100E300083F3118862B6704702684368114301600A
:100E400003B118477047000013B5446BD4F89434CD
:100E50001A681178042915D1217C022912D1197937
:100E6000128901238B4013420CD101A904F14C00DB
:100E700001F05CFED4F89444019B2179024620687D
:100E800000F0E6F902B010BD143001F0E1BD000041
:100E90004FF0FF33143001F0DBBD00004C3001F0A7
:100EA000B1BE00004FF0FF334C3001F0ABBE00008C
:100EB000143001F0B1BD00004FF0FF31143001F0EB
:100EC000ABBD00004C3001F07DBE00004FF0FF32A2
:100ED0004C3001F077BE0000D0F8942438B5136888
:100EE00019780429054601D0012038BD017C02296A
:100EF000FAD112795C89012090400440F4D105F1C7
:100F0000140001F043FD02460028EDD0D5F89454BA
:100F10004FF480732868697900F088F9204638BD5D
:100F2000406BFFF7D9BF00000020704770470000FA
:100F30007FB5124B0360002343608360C3600125CB
:100F400002260F4B057404460290019300F18402BF
:100F5000294600964FF48073143001F0F3FC094BDE
:100F60000193029400964FF4807304F5237229468E
:100F700004F14C0001F0B6FD04B070BD043400086B
:100F8000210F0008490E000808B50A68FFF74EFF58
:100F90000B7902EB830318624B790D3342F823007F
:100FA0008B7913B102EB8302106202230374C0F841
:100FB0009414002383F3118808BD000038B5037F23
:100FC000044613B190F85430ABB9201D012502211D
:100FD000FFF732FF04F1140025776FF0010100F0F4
:100FE00095FC84F8545004F14C006FF00101BDE809
:100FF000384000F08BBC38BD10B5012104460430E8
:10100000FFF71AFF0023237784F8543010BD000047
:1010100038B504460025143001F0ACFC04F14C0056
:10102000257701F077FD201D84F854500121FFF74A
:1010300003FF2046BDE83840FFF74EBF90F85C3014
:1010400003F06003202B19D190F85D20212A0AD0EB
:10105000222A4FF000030ED0202A0FD1084A026541
:101060000722426504E0064B03650723436500231E
:1010700083650120704703654365F9E700207047E9
:1010800028240120D0F8943437B51A68117804293F
:1010900004461AD1017C022917D11979128901233A
:1010A0008B40134211D100F14C05284601F0F0FDB0
:1010B00058B101A9284601F039FDD4F89444019BA8
:1010C00021790246206800F0C3F803B030BD00006B
:1010D00000EB8103F7B51C6A05460E46ECB105EB43
:1010E0008607FFF7A3FE201D0821FFF7A5FEFB687A
:1010F0005B691B684C3413B1204601F025FD01A942
:10110000204601F013FD024648B1019B31462846B6
:1011100000F09EF8002383F3118803B0F0BDFB6854
:101120005A691268002AF5D01B8A013B1340F1D19D
:1011300005F15C02EAE700000D3138B550F82140B6
:10114000D4B1FFF773FED4F894241368527903EBFB
:101150008203DB689B695D6845B104216018FFF775
:101160006BFE294604F1140001F01AFC2046FFF73B
:10117000B3FE002383F3118838BD000070470000E0
:1011800072B6202383F3118862B6704700F0A0BFC7
:10119000012303700023436000F1240200F13801B1
:1011A00042F8043B8A421361FAD1038143817047BC
:1011B00038B50446FFF7E4FF00254160C5600561CE
:1011C00045618561C561056200F092FF02232370CD
:1011D00085F3118838BD000070B500EB810305462A
:1011E0005069DA600E46144618B110220021FFF74C
:1011F000DFFDA06918B110220021FFF7D9FD3146AB
:101200002846BDE8704001F03DB80000028902F0B8
:1012100001020281428902F0010242810022026140
:1012200042618261C261026201F0C0B8F0B400EBB9
:1012300081044789E4680125A4698D403D434581C7
:1012400023600023A2606360F0BC01F0DBB8000003
:10125000F0B400EB81040789E468012564698D40DE
:101260003D43058123600023A2606360F0BC01F070
:1012700057B9000070B50223002504460370A0F89A
:10128000645080F8665080F8675005814581C560DC
:10129000056145618561C561056280F84C5000F0CB
:1012A0008DFF63681B6823B129462046BDE8704066
:1012B000184770BD436802781B6880F868200522D3
:1012C00002700BB10421184770470000436890F882
:1012D00068201B6802700BB1052118477047000099
:1012E00090F84C3070B5044613B1002380F84C30B0
:1012F00004F15C02204601F07BF863689B6863BBE5
:1013000094F85C5015F0600615D194F85D3005F046
:101310007F0545EA032540F202339D4200F00B8130
:1013200059D8022D00F0D9803DD8002D00F08580DD
:10133000012D00F0CC800021204601F0C9FA0021E7
:10134000204601F0BBFA63681B6813B106212046F2
:101350009847062384F84C3070BD204698470028F3
:10136000CED094F8632094F8623043EA0223626D91
:10137000934238BF636594F95C30656D002B80F251
:10138000FC80002D00F0EB80092384F84C30FFF73F
:10139000F7FE636D226D00212046FFF759FF002301
:1013A00083F3118870BDB5F5817F00F0B080B5F58D
:1013B000407F49D0B5F5807FBDD194F85E30012BD8
:1013C000B9D1B4F8643023F00203A4F86430266580
:1013D0006665A665C5E740F201639D421ED8B5F576
:1013E000C06F3BD2B5F5A06FA5D1B4F85C30B3F5B2
:1013F000A06F0ED194F85E3084F86630204600F07D
:1014000035FF63681B6813B1012120469847032309
:101410002370002323656365A365A2E7B5F5106F0C
:1014200032D040F602439D4251D0B5F5006F82D1D3
:1014300004F167032365012324E004F164032365B9
:1014400002236365A5658CE794F85E30012B7FF479
:1014500072AFB4F8643043F00203B6E794F8612049
:10146000616894F860304D6894F85F1043EA022395
:10147000204694F85E20A84700283FF45CAF4368FC
:10148000236503686365A4E72378042B0FD1FFF776
:1014900077FE2046FFF7BAFE86F31188636884F86A
:1014A00067601B68032121700BB12046984794F8B0
:1014B0005E30002BADD084F867300423237063685E
:1014C0001B68002BA5D0022120469847A1E7374B87
:1014D00023650223636500239EE794F8601011F0F2
:1014E000800F204601F00F010ED000F073FF01289D
:1014F00006D002287FF41FAF2D4B2365606568E797
:101500002C4B2365656564E700F056FFEFE794F820
:101510005E30002B7FF40FAF94F8603013F00F01B2
:101520003FF477AF1A06204602D501F0E5F970E7DF
:1015300001F0D8F96DE794F85E30002B7FF4FBAE34
:1015400094F8603013F00F013FF463AF1B062046A0
:1015500002D501F0BDF95CE701F0B0F959E71423B9
:1015600084F84C30FFF70CFE2B462A4629462046CD
:10157000FFF75CFE85F3118870BD5DB1152384F81B
:101580004C30FFF7FDFD636D226D00212046FFF713
:101590004DFE04E70B2384F84C30FFF7F1FD2B469A
:1015A0002A4629462046FFF753FEE3E73434000875
:1015B0002C3400083034000838B590F84C3004461C
:1015C000152B28D8DFE803F03C27272727273C27BF
:1015D000270B283727272727272727273C3C90F842
:1015E000631090F86220436D42EA01229A4213D9B7
:1015F000C268128AB3FBF2F502FB153565B9FFF735
:10160000BFFD2B462A462946FFF722FE85F31188A7
:101610000A2384F84C3038BD142384F84C30FFF78B
:10162000AFFD00231A4619462046FFF7FFFD0023B1
:1016300083F3118838BD836D03B198470023E8E731
:10164000002101F045F90021204601F037F96368D7
:101650001B6813B10621204698470623D9E70000EE
:1016600090F84C20152A38B5044621D80123934020
:1016700040F6416213421CD113F480150ED19B0237
:1016800016D50B2380F84C30FFF77AFD2B462A46FF
:101690002946FFF7DDFD85F3118838BDC3689B69D6
:1016A0005B682BB9836D03B19847002384F84C30F5
:1016B00038BD002101F00CF90021204601F0FEF8B0
:1016C00063681B6813B10621204698470623EDE79F
:1016D000024B00221B605B609A607047B0290120BA
:1016E000002303748268054B1B6899689142FBD202
:1016F0005A6803604260106058607047B02901204A
:1017000008B572B6202383F3118862B6037C032BDD
:1017100005D0042B0DD02BB983F3118808BD436984
:1017200000221A604FF0FF334361FFF7D9FF002317
:10173000F2E790E80C001A6002685360F2E70000DC
:10174000002303748268054B1B6899689142FBD89B
:101750005A6803604260106058607047B0290120E9
:10176000054B19690874186802681A60536018619B
:1017700001230374FEF7D8BDB029012030B54B1CFE
:1017800087B005460A4C10D023690A4A01A800F028
:10179000D9F82846FFF7E4FF049B13B101A800F035
:1017A0000DF92369586907B030BDFFF7D9FFF8E795
:1017B000B02901200117000838B50C4D41612B6993
:1017C00081689A689142044603D8BDE83840FFF723
:1017D00087BF1846FFF784FF01232C61014623745D
:1017E0002046BDE83840FEF79FBD00BFB02901206C
:1017F000044B1A681B6990689B68984294BF00204C
:1018000001207047B029012010B5084C23682069D9
:101810001A6822605460012223611A74FFF790FF56
:1018200001462069BDE81040FEF77EBDB0290120C9
:1018300072B6202383F3118862B670478260022259
:1018400002740022427470478368A3F17C0243F85B
:101850000C2C026943F83C2C426943F8382C074AA7
:1018600043F81C2CC26843F8102C022203F8082C01
:10187000002203F8072CA3F1180070474103000869
:1018800010B5FFF7D5FFFFF7DFFF00210446FFF794
:1018900093FF002383F31188204610BD024B1B6980
:1018A00058610F20FFF75CBFB029012008B5FFF792
:1018B000BFFFBDE80840FFF7F1BF000008B50146D3
:1018C000FFF7B6FF0820FFF759FF002383F31188C5
:1018D00008BD000049B1064B42681B6918605A6098
:1018E000136043600420FFF749BF4FF0FF3070479B
:1018F000B02901200368984206D01A68026050603F
:1019000059611846FFF7ECBE7047000038B5044631
:101910000D462068844200D138BD036823605C60B6
:101920004561FFF7DDFEF4E7054B03F114025A6150
:101930009A614FF0FF32DA6100221A62704700BFED
:10194000B0290120F8B503614FF08043C2605C6AA2
:10195000194B1A46022952F8145F38BF02219542EA
:1019600006461F460AD1586198611C6205604560B1
:1019700081600819BDE8F84001F0ACB9186AAB689D
:10198000241A0C1902D3E41A2D6804E09C4202D2F6
:10199000204401F0ADF9AB689C42F4D86B687360E9
:1019A00035601E606E60B460A9684FF0FF33091B9C
:1019B000A960FB61F8BD00BFB029012010B41B4C29
:1019C000234653F8141F814210D0416802680A6010
:1019D000026851609A424FF00001C16003D09368E1
:1019E00081680B4493605DF8044B70470A6862613C
:1019F00000209A425360C86003D15DF8044B01F0A7
:101A000071B993688868034493604FF08042206AFC
:101A1000526A121A9342E6D9991A012998BF931C67
:101A200018445DF8044B01F063B900BFB0290120F0
:101A300000207047FEE70000704700004FF0FF30C5
:101A40007047000072B6202383F3118862B6704796
:101A5000022906D0032906D00129064818BF002014
:101A6000704705487047032A9ABF044800EBC2003C
:101A7000002070472C350008E03400083024012095
:101A800070B5044608460D46FFF78AF9C6B22046EF
:101A9000013403780BB9184670BD32462946FFF76A
:101AA00067F90028F3D1012070BD00002DE9F04F47
:101AB00081469BB008460D461646FFF771F93D4931
:101AC000C4B22846FFF7DCFF08B10434E4B23A4957
:101AD0002846FFF7D5FF08B11034E4B2632C01AFFC
:101AE0000CD8DFF8E0A0DFF8E0B03C4695F80080C5
:101AF000B8F1000F1CD184F8008003E02946384675
:101B000001F05EFC3846FFF74BF9C0B2431C5B00A6
:101B100089E84800337003237370002302361946A6
:101B2000DAB2904206F102063DD81BB0BDE8F08F54
:101B3000B8F1250F32D107221E492846FFF718F9C0
:101B400070B9DBF800202260DBF804206260BBF88B
:101B5000082022819BF80A20A27207350B34C5E7C2
:101B6000082215492846FFF703F9B8B91348A21C03
:101B700010F8011F124B4FEA111E01F00F011EF861
:101B80000AE011F80A1002F802EC984202F8011C6F
:101B900002F10202ECD118340835A7E784F800807E
:101BA00001350134A2E7FA5C06F8022C06F8011CA4
:101BB0000133B5E788340008903400081FF4F01FA3
:101BC0002BF4F01FA53400089934000808B5FFF77E
:101BD00039FF0348FFF756FA002383F3118808BD45
:101BE000F029012010B50446052915D8DFE801F0D9
:101BF00015140315151BFFF725FF0E4A0121FFF7EA
:101C0000EBFA20460C4A0221FFF7E6FA0B48FFF7F1
:101C1000FFF9002383F3118810BDFFF713FF074876
:101C2000FFF7CCF9F5E7FFF70DFF0448FFF7E4F9FC
:101C3000EFE700BF383400085C340008F0290120C9
:101C400038B50C4D0C4C0D492A4604F10800FFF73D
:101C50002DFF05F1CA0204F110000949FFF726FF24
:101C600005F5CA7204F118000649BDE83840FFF7CF
:101C70001DBF00BFB82E012030240120B834000859
:101C8000C234000890340008BFF34F8F024AD36873
:101C9000DB03FCD4704700BF003C024008B5074B93
:101CA0001B7853B9FFF7F0FF054B1A69002ABFBF35
:101CB000044A5A6002F188325A6008BD1631012088
:101CC000003C02402301674508B5054B1B7833B93A
:101CD000FFF7DAFF034A136943F00043136108BDBD
:101CE00016310120003C0240072870B513D80B4A7A
:101CF0000B4C137863B90B4E4FF0006144F823107E
:101D000056F823500133082B2944F7D101231370CF
:101D100054F8200070BD002070BD00BF3831012094
:101D2000183101204C350008014B53F82000704752
:101D30004C35000808207047072810B5044601D923
:101D4000002010BDFFF7D0FF064B53F82430184495
:101D5000C21A0BB9012010BD12680132F0D1043B48
:101D6000F6E700BF4C350008072810B504462FD809
:101D7000FFF78AFFFFF792FF1649F323CB60FFF7C7
:101D800083FFC300DBB243F4007343F002030B6133
:101D90000B6943F480330B61FFF776FFFFF7A4FF75
:101DA0000D4B53F824300344BFF34F8F0B4A984236
:101DB0000AD3BFF34F8FBFF36F8FFFF785FF204626
:101DC000BDE81040FFF7B8BFC2F85C022030EEE774
:101DD000002010BD003C02404C35000800ED00E042
:101DE0002DE9F84312F00103154643D10244B2F144
:101DF000016F3FD22C4B1B6813F001033AD02B4CE0
:101E0000FFF74CFFF323E360FFF73EFF40F20127AB
:101E1000032D16D8254C0F46401A40F20118EB1B33
:101E20000B44012B00EB0706236926D823F001039E
:101E30002361FFF749FF0120BDE8F883043D04302A
:101E4000E6E78307E6D1236923F44073236123691E
:101E50003B43236151F8046B0660BFF34F8FFFF7DC
:101E600013FF03689E42E9D0236923F00103236135
:101E7000FFF72AFF0020BDE8F88323F440732361B5
:101E8000236943EA08032361B94637F8023B3380EC
:101E9000BFF34F8FFFF7F8FE3688B9F80030B6B2BF
:101EA000B342BCD0E0E700BF00380240003C024033
:101EB000084908B50B7828B153B9FFF7EFFE0123A5
:101EC0000B7008BD23B1BDE808400870FFF7FCBEE9
:101ED00008BD00BF16310120014B186D704700BFCF
:101EE00000280040094B1A6F120407D41A6F42F4FD
:101EF00000721A671A6F42F400421A67044A1368A4
:101F000043F480731360034B186570470038024038
:101F10000070004000280040034B1B689B0042BF3C
:101F2000024B01221A707047743802403931012087
:101F3000014B1878704700BF39310120F0B5BFF36D
:101F40004F8FBFF36F8F1D4B0021C3F85012BFF3AB
:101F50004F8FBFF36F8F5A6942F400325A61BFF35B
:101F60004F8FBFF36F8FC3F88410BFF34F8FD3F839
:101F70008020C2F3C904C2F34E325201A50743F6D2
:101F8000E07602EA060E284621464EEA00070139AD
:101F9000C3F860724F1C00F14040F6D1203A12F1B4
:101FA000200FEED1BFF34F8F5A6942F480325A614D
:101FB000BFF34F8FBFF36F8FF0BD00BF00ED00E0A8
:101FC000FEE70000084A094B09498B4204D3094A3D
:101FD0000021934205D3704752F8040F43F8040BD5
:101FE000F3E743F8041BF4E74437000848340120C2
:101FF0004834012048340120036F30B500229D6829
:10200000C46E11464FF0FF3004EB4213013295428B
:10201000C3F80019C3F81019C3F80809C3F8001B66
:10202000C3F8101BC3F8080BEED24FF00113C4F82D
:102030001C3830BD890141F02001016103699B0614
:10204000FCD4122000F0E4BE204B03EB80022DE90B
:10205000F047D2F80CE0DD6EDEF81420461CD2F812
:1020600000C005EB063605EB4018516861450BD3FF
:10207000D5F83428012303FA00F022EA0000C5F85D
:1020800034081846BDE8F087BEF81040ACEB0103F9
:10209000A34228BF2346D8F81849A4B2B3EB840F53
:1020A00010D894681F46A4F1040959F804AFC6F883
:1020B00000A0042F01D9043FF7E71C440B449460AF
:1020C0005360D2E70020BDE8F08700BF3C3101201B
:1020D00010B5054C2046FFF75BF84FF0A043E366D0
:1020E000024B236710BD00BF3C3101209035000832
:1020F0000378012B70B5054650D12A4BC46E984227
:102100001BD1294B5A6B42F080025A635A6D42F040
:1021100080025A655A6D5A6942F080025A615A69C2
:1021200022F080025A610E2143205B6900F0EEFB31
:102130001E4BE3601E4BC4F800380023C4F8003E79
:10214000C0232360EE6E4FF40413A3633369002BA6
:10215000FCDA012333610C2000F05AFE3369DB07FF
:10216000FCD4122000F054FE3369002BFCDA002668
:10217000A6602846FFF740FF6B68C4F81068DB686C
:10218000C4F81468C4F81C684BB90A4BA3614FF03B
:10219000FF336361A36843F00103A36070BD064B86
:1021A000F4E700BF3C3101200038024040140040F9
:1021B00003002002003C30C0083C30C0F8B5C46EBB
:1021C000054600212046FFF735FF296F00234FF019
:1021D00001128F68C4F834384FF00066C4F81C2828
:1021E0004FF0FF3004EB431201339F42C2F8006905
:1021F000C2F8006BC2F80809C2F8080BF2D20B68EB
:10220000EA6E6B67636210231361166916F010069D
:10221000FBD1122000F0FCFDD4F8003823F4FE635B
:10222000C4F80038A36943F4402343F01003A361CA
:102230000923C4F81038C4F814380A4BEB604FF087
:10224000C043C4F8103B084BC4F8003BC4F8106905
:10225000C4F800396B6F03F1100243F480136A670E
:10226000A362F8BD6C35000840800010C26E90F883
:102270006610D2F8003823F4FE6343EA0113C2F873
:10228000003870472DE9F0410EB200EB86080D468C
:10229000D8F80C100F6807F00303022B50D0032B63
:1022A00050D03D4A3D4F012B18BF1746C46E4FEA30
:1022B000451E04EB0E030022C3F8102B8A6905F1BA
:1022C000100C002A40D04A8A05F158035B013A43BA
:1022D000E2500123D4F81C2803FA0CF31343A6445C
:1022E0004A69C4F81C380023CEF8103905F13F03C1
:1022F000002A39D00A8A898B9208012988BF4A436B
:10230000416F04EB8303561841EA024246672946AF
:102310005A602046FFF78EFED8F80C301B8A43EA3D
:1023200085531F4305F148035B01E7500123D4F8AF
:102330001C2803FA05F51543C4F81C58BDE8F081C4
:10234000174FB3E7174FB1E704EB4613D3F8002B51
:1023500022F40042C3F8002BD4F81C28012303FA0E
:102360000CF322EA0303BAE704EB83030E4A5A6034
:1023700004EB461629462046FFF75CFED6F80039E6
:1023800023F40043C6F80039D4F81C38012202FABD
:1023900005F523EA0505CFE7008000100080041052
:1023A0000080081000800C1000040002026F126808
:1023B0004267FFF721BE00005831C36E49015B58E8
:1023C00013F4004004D013F4001F14BF01200220B6
:1023D000704700004831C36E49015B5813F4004058
:1023E00004D013F4001F14BF012002207047000026
:1023F00000EB8101CB68196A0B6813604B6853606E
:102400007047000000EB810330B5DD68AA691368EE
:10241000D36019B9402B84BF402313606B8A1468C2
:10242000C26E1C44013CB4FBF3F46343033323F05A
:10243000030302EB411043EAC44343F0C043C0F836
:10244000103B2B6803F00303012B09B20ED1D2F825
:10245000083802EB411013F4807FD0F8003B14BF22
:1024600043F0805343F00053C0F8003B02EB4112AD
:10247000D2F8003B43F00443C2F8003B30BD0000FB
:102480002DE9F041254DEE6E06EB40130446D3F8DE
:10249000087BC3F8087B38070AD5D6F81438190723
:1024A00006D505EB84032146DB6828465B68984720
:1024B000FA0731D5D6F81438DB072DD505EB8403A0
:1024C000D968DCB98B69488A5E68B6FBF0F200FB1C
:1024D00012629AB91868DA6890420FD2121A83E829
:1024E000140072B6202383F3118862B60B4821468C
:1024F000FFF788FF84F31188BDE8F081012303FA18
:1025000004F26B8923EA02036B81CB6823B1214675
:102510000248BDE8F0411847BDE8F0813C31012098
:1025200000EB810370B5DD68C36E6C692668E660F8
:102530004A0156BB1A444FF40020C2F810092A6819
:1025400002F00302012A0AB20ED1D3F8080803EB05
:10255000421410F4807FD4F8000914BF40F080507A
:1025600040F00050C4F8000903EB4212D2F8000911
:1025700040F00440C2F80009D3F83408012202FAFE
:1025800001F10143C3F8341870BD19B9402E84BF5E
:102590004020206020682E8A841940F00050013CC1
:1025A0001A44B4FBF6F440EAC440C6E7F8B5044662
:1025B0001F48C56E05EB4413D3F80869C3F80869D2
:1025C000F10719D5D5F81038DA0715D500EB8403D3
:1025D000D9684B691F68DA6897421AD2D21B002764
:1025E0001A605F6072B6202383F3118862B62146B9
:1025F000FFF796FF87F31188330617D5D5F83428EF
:102600000123A340134211D02046BDE8F840FFF754
:102610001BBD012303FA04F2038923EA02030381A9
:102620008B68002BE8D021469847E5E7F8BD00BF4E
:102630003C310120A0482DE9F84FC56E6E69AB69A9
:102640001E4016F4805F6E61044605D0FEF712FE50
:10265000BDE8F84F00F07EBC002E12DAD5F8003E3F
:1026600095489B071EBFD5F8003E23F00303C5F82D
:10267000003ED5F8043823F00103C5F80438FEF70E
:1026800025FE370502D58C48FEF714FEB0040CD5A4
:10269000D5F8083813F0060FEB6823F470530CBF1D
:1026A00043F4105343F4A053EB60310704D563683F
:1026B000DB680BB180489847F2026FD4B3020CD5A7
:1026C000D4F86C80DFF8F0A100274FF00109236FE8
:1026D0009B68F9B28B4280F09C80F70619D5E16EB9
:1026E0000A6AC2F30A1702F00F0302F4F012B2F5FD
:1026F000802F00F0B680B2F5402F0AD104EB83039F
:1027000001F58051DB68186A00231A469F4240F0A9
:102710009C803303D5F818481DD5E70302D5002067
:10272000FFF7AEFEA50302D50120FFF7A9FE600367
:1027300002D50220FFF7A4FE210302D50320FFF7F4
:102740009FFEE20202D50420FFF79AFEA30202D503
:102750000520FFF795FE77037FF57AAFE60702D5F0
:102760000020FFF723FFA50702D50120FFF71EFF7A
:10277000600702D50220FFF719FF210702D50320C9
:10278000FFF714FFE20602D50420FFF70FFFA306B0
:102790007FF55EAF0520FFF709FF59E7D4F86C809D
:1027A000DFF814A100274FF00109236F9B685FFA3F
:1027B00087FB5B4582D308EB4B13D3F8002902F467
:1027C0004022B2F5802F22D1D3F80029002A1EDA48
:1027D000D3F8002942F09042C3F80029D3F8002929
:1027E000002AFBDB5946E06EFFF724FC228909FA38
:1027F0000BF322EA0303238104EB8B03DB689B6862
:1028000013B15946504698475846FFF71DFC01370B
:10281000CBE708EB4112D2F8003B03F44023B3F5B9
:10282000802F10D1D2F8003B002B0CDA628909FA14
:1028300001F322EA0303638104EB8103DB68DB68B5
:102840000BB150469847013741E79C0708BF0A681B
:10285000072B98BF027003F101039CBF120A0130DD
:1028600054E7023304EB830201F58051526890690A
:102870000268D0F808C04068A2EB000E00221046A3
:1028800097420AD104EB830463689B699A683A44CF
:102890009A605A6817445F603BE712F0030F08BF65
:1028A0000868964588BF8CF8000002F1010284BFD9
:1028B000000A0CF1010CE3E73C310120C36E03EB8D
:1028C0004111D1F8003B43F40013C1F8003B7047BD
:1028D000C36E03EB4111D1F8003943F40013C1F882
:1028E00000397047C36E03EB4111D1F8003B23F46C
:1028F0000013C1F8003B7047C36E03EB4111D1F8E0
:10290000003923F40013C1F80039704700F1604327
:1029100000F01F02400903F5614309018000C9B2BC
:1029200000F1604083F8001300F5614001239340FB
:10293000C0F880310360704772B6202383F311889A
:1029400062B6704730B5039C0172043304FB032563
:10295000C361049B03630021059B00604060C1606C
:10296000426102618561046242628162C1624363C5
:1029700030BD00000022416A41610161C260826293
:10298000C2626FF00101FEF7C1BF00000369426936
:10299000934203D1C2680AB100207047181D7047E6
:1029A00003691960C2680132C260C2691344826956
:1029B0000361934224BF436A03610021FEF79ABF7B
:1029C00038B504460D46E3683BB16269131D1268D1
:1029D000A3621344E362002038BD237A33B9294649
:1029E0002046FEF777FF0028EDDA38BD6FF00100D2
:1029F000FBE70000C368C269013BC360436913443D
:102A000082694361934224BF436A43610023836226
:102A1000036B03B11847704770B50446FFF78CFF8E
:102A2000866A3EB9FFF7CCFF054618B186F31188D8
:102A3000284670BDA36AE26A13F8015BA362934261
:102A400002D32046FFF7D6FF002383F31188EFE778
:102A50002DE9F04704460E4617469846FFF76CFFEF
:102A60000025A946D4F828A0BAF1000F09D14146A3
:102A70002046FFF7A5FF20B18AF311882846BDE85C
:102A8000F087A16AE36AA7EB050A5B1A9A4528BF9B
:102A90009A46BAF1400F1BD9334601F1400251F872
:102AA000040B43F8040B9142F9D1A36A403340363A
:102AB000A3624035A26AE36A9A4202D32046FFF736
:102AC00099FF89F31188BD42D8D2FFF735FFC9E7D6
:102AD00030465246FEF742F9A36A53445644A36275
:102AE0005544E7E710B5029C0172043303FB04214F
:102AF000C36100238362C362039B0363049B006082
:102B00004060C46042610261816104624262436369
:102B100010BD0000026AC260426A42610261002286
:102B20008262C2626FF00101FEF7F0BE4369026982
:102B30009A4203D1C2680AB100207047184650F883
:102B4000043B0B6070470000C368C2690133C36077
:102B50004369134482694361934224BF436A4361DA
:102B60000021FEF7C7BE000038B504460D46E368F5
:102B70003BB123691A1DA262E2691344E36200209B
:102B800038BD237A33B929462046FEF7A3FE002834
:102B9000EDDA38BD6FF00100FBE700000369196052
:102BA000C268013AC260C2691344826903619342F8
:102BB00024BF436A036100238362036B03B1184798
:102BC0007047000070B504460E46FFF7B5FE856AF3
:102BD00035B91146FFF7C8FF10B185F3118870BDF4
:102BE000A36A1E70A36AE26A01339342A36204D30C
:102BF000E16920460439FFF7D1FF002080F31188F6
:102C000070BD00002DE9F04704460D4690469946F8
:102C1000FFF792FE0026B246A76A4FB94946204602
:102C2000FFF7A2FF20B187F311883046BDE8F08797
:102C3000A06AE76AA8EB06033F1A9F4228BF1F4617
:102C4000402F1BD905F1400355F8042B40F8042B05
:102C50009D42F9D1A36A4033A3624036A26AE36A77
:102C60009A4204D3E16920460439FFF797FF8AF3BB
:102C700011884645D9D2FFF75FFECDE729463A468F
:102C8000FEF76CF8A36A3B443D44A3623E44E5E78B
:102C9000026943699A4203D1C3681BB91846704759
:102CA0000023FBE7836A002BF8D0043B9B1AF5D086
:102CB0001360C368013BC360C3691A44836902613E
:102CC0009A4224BF436A0361002383620123E5E73C
:102CD00000F086B94FF08043002258631A61022247
:102CE000DA6070474FF080430022DA6070470000DE
:102CF0004FF0804358637047FEE7000010B5194C51
:102D0000FEF7E6FCFEF710FE802217492046FEF78C
:102D100095FD012344F8180C0374144B144AD96828
:102D200021F4E0610904090C0A431249DA60CA6817
:102D300042F08072CA60104A1049C2F8B01F116890
:102D400041F0010111601022DA77202283F822205D
:102D5000002383F3118862B60948BDE81040FEF7EE
:102D60008FBD00BFD82901209C35000800ED00E090
:102D70000003FA05F0ED00E0001000E055CEACC510
:102D8000A43500082DE9F84F204C4FF00008656984
:102D900004F11407C1464FF08043266A5B6AAA68B3
:102DA0009E1B96421FD34FF0200AAA68236AD5F8CB
:102DB0000CB0134423622B68BB425F60A6EB020693
:102DC0006361C5F80C8001D1FFF78CFF89F311888E
:102DD0002869D84772B68AF3118862B66569AB680C
:102DE0009E42E2D2D7E76269BA420CD09168236270
:102DF0008E1B9660A86802282CBF1818981CBDE886
:102E0000F84FFFF775BFBDE8F88F00BFB02901206C
:102E1000034B59685A68521A9042FBD8704700BF5A
:102E2000001000E04B6843608B688360CB68C36030
:102E30000B6943614B6903628B6943620B680360F2
:102E40007047000008B5274B27481A6940F2FF7108
:102E50000A431A611A6922F4FF6222F007021A611A
:102E60001A691A6B0A431A631A6D0A431A651F4AD4
:102E70001B6D1146FFF7D6FF1D4802F11C01FFF73D
:102E8000D1FF1C4802F13801FFF7CCFF1A4802F1CC
:102E90005401FFF7C7FF194802F17001FFF7C2FFA5
:102EA000174802F18C01FFF7BDFF164802F1A80197
:102EB000FFF7B8FF144802F1C401FFF7B3FF13484E
:102EC00002F1E001FFF7AEFF114802F1FC01FFF74C
:102ED000A9FF104802F58C71FFF7A4FFBDE8084078
:102EE00000F0E0B80038024000000240C43500089D
:102EF0000004024000080240000C024000100240A2
:102F00000014024000180240001C02400020024051
:102F1000002402400028024008B500F035FAFFF70F
:102F2000EDFEFEF7F9FFBDE80840FEF789BE0000A0
:102F300070470000064A536823F001035360EFF323
:102F40000983683383F30988002383F3118870476A
:102F500030EF00E010B572B6202383F3118862B61B
:102F6000104B5B6813F4006318D0F1EE103AEFF3E6
:102F700009844FF0807344F84C3C0B4BDB6844F8F9
:102F8000083CA4F1680383F30988FEF731FC18B10B
:102F9000064B44F8503C10BD054BFAE783F311880B
:102FA00010BD00BF00ED00E030EF00E0510300086D
:102FB000540300084FF0804310B51A6992070AD5F0
:102FC00000241C6172B6202383F3118862B6FFF7D8
:102FD000D9FE84F31188BDE81040FFF7BBBF0000A5
:102FE000104B1A6C42F001021A641A6E42F0010290
:102FF0001A660D4A1B6E936843F0010393604FF00D
:1030000080436B229A624FF0FF32DA6200229A61AB
:103010005A63DA605A6001225A6108211A601C2042
:10302000FFF774BC00380240002004E01B4B1A6913
:103030006FEA42526FEA52521A611A69C2F30A02E7
:103040001A614FF0FF301A695A69586100215A69B4
:1030500059615A691A6A62F080521A621A6A02F059
:1030600080521A621A6A5A6A58625A6A59625A6ACD
:103070000B4A106840F480701060186F00F44070C4
:10308000B0F5007F1EBF4FF4803018671967536892
:1030900023F40073536000F057B900BF00380240BA
:1030A00000700040354B4FF080521A64344A4FF4A0
:1030B000404111601A6842F001021A601A689207D2
:1030C000FCD59A6822F003029A602C4B19469A6844
:1030D00012F00C02FBD1186800F0F90018609A6039
:1030E0001A6842F480321A600B689B03FCD54B6F60
:1030F00043F001034B67214B5A6F9007FCD5214ADF
:103100005A601A6842F080721A601D4B1A4659685C
:103110004904FCD5196841F4803119605368D8031B
:10312000FCD5136843F400331360154A53689903C0
:10313000FCD5124B1A689201FCD5134A9A6040F2F2
:103140000112C3F88C200022C3F890200F4A40F2ED
:10315000073111609A6842F002029A60074B9A6840
:1031600002F00C02082AFAD15A6C42F480425A64E6
:103170005A6E42F480425A665B6E704700380240D5
:1031800000700040086C400900948838003C024000
:10319000084A08B5536911680B4003F001035361F5
:1031A00023B1054A13680BB150689847BDE8084041
:1031B000FFF7D0BE003C0140C8330120084A08B5E3
:1031C000536911680B4003F00203536123B1054AB0
:1031D00093680BB1D0689847BDE80840FFF7BABEC6
:1031E000003C0140C8330120084A08B55369116802
:1031F0000B4003F00403536123B1054A13690BB17B
:1032000050699847BDE80840FFF7A4BE003C014064
:10321000C8330120084A08B5536911680B4003F010
:103220000803536123B1054A93690BB1D0699847EC
:10323000BDE80840FFF78EBE003C0140C8330120C6
:10324000084A08B5536911680B4003F01003536135
:1032500023B1054A136A0BB1506A9847BDE808408C
:10326000FFF778BE003C0140C8330120174B10B572
:103270005C691A68144004F478725A61A30604D594
:10328000134A936A0BB1D06A9847600604D5104A76
:10329000136B0BB1506B9847210604D50C4A936B06
:1032A0000BB1D06B9847E20504D5094A136C0BB1FA
:1032B000506C9847A30504D5054A936C0BB1D06CAC
:1032C0009847BDE81040FFF745BE00BF003C0140F5
:1032D000C83301201A4B10B55C691A68144004F415
:1032E0007C425A61620504D5164A136D0BB1506DCC
:1032F0009847230504D5134A936D0BB1D06D9847B9
:10330000E00404D50F4A136E0BB1506E9847A10428
:1033100004D50C4A936E0BB1D06E9847620404D565
:10332000084A136F0BB1506F9847230404D5054A20
:10333000936F0BB1D06F9847BDE81040FFF70ABEFE
:10334000003C0140C8330120062108B50846FFF7BC
:10335000DDFA06210720FFF7D9FA06210820FFF73A
:10336000D5FA06210920FFF7D1FA06210A20FFF736
:10337000CDFA06211720FFF7C9FA06212820BDE85B
:103380000840FFF7C3BA000008B5FFF74FFE00F092
:103390000BF8FDF7FBFEFDF7C9FDFFF7C9FDBDE822
:1033A0000840FFF795BC0000002304491A465A5014
:1033B000C8180833802B4260F9D17047C833012008
:1033C000034611F8012B03F8012B002AF9D17047AD
:1033D000121012131211000053544D3332463F3F66
:1033E0003F3F3F3F0053544D333246375B347C35CB
:1033F0005D780053544D333246375B367C375D7809
:103400000000000000000000A50E0008910E00085A
:10341000CD0E0008B90E0008C50E0008B10E000858
:103420009D0E0008890E0008290F0008000000000A
:103430000100000000000000020000000000000089
:10344000D11000083911000840004000882E0120EA
:10345000982E012002000000000000000300000080
:10346000000000007D1100080000000010000000B6
:10347000A82E012000000000010000000000000054
:103480003C3101200101020025424F4152442500F8
:103490002553455249414C25004F4D4E4942555305
:1034A00046375632003031323334353637383941C9
:1034B00042434445460000004172647550696C6F98
:1034C000740025424F415244252D424C000000001B
:1034D000E51B0008511A00083D100008CD1B00082C
:1034E00043000000E834000809024300020100C064
:1034F0003209040000010202010005240010010548
:1035000024010001042402020524060001070582AB
:10351000030800FF09040100020A0000000705017A
:103520000240000007058102400000001200000078
:103530003435000812011001020000408304405796
:1035400000020102030100000403090400800000DE
:1035500000800000008000000080000000000200E9
:10356000000004000000040000000400000000004F
:10357000E1120008B915000861160008400040007B
:10358000B4310120B431012001000000C431012018
:103590008000000040010000050000006D61696EC0
:1035A00000000000BC350008D0310120C8330120E4
:1035B00001000000F92C00080000000069646C653F
:1035C000000000001000802A00000000AAAAAAAA99
:1035D00000000000FFFF00000000000000A00A0043
:1035E0000000000000000000AAAAAAAA0000000033
:1035F000FFFF0000000000000000000000000000CD
:1036000000000000AAAAAAAA00000000FFFF000014
:1036100000000000000000000000000000000000AA
:10362000AAAAAAAA00000000FFFF000000000000F4
:10363000000000000000000000000000AAAAAAAAE2
:1036400000000000FFFF000000000000000000007C
:103650000000000000000000AAAAAAAA00000000C2
:10366000FFFF00000000000000000000000000005C
:1036700000000000AAAAAAAA00000000FFFF0000A4
:10368000000000000000000000000000000000003A
:103690000A0000000000000003000000000000001D
:1036A000000000000000000000000000000000001A
:1036B000000000000000000000000000000000000A
:1036C00000000000000000000000000000000000FA
:1036D00000000000000000000000000000000000EA
:1036E00000000000000000000000000000000000DA
:1036F0000000000000000000FF00000000000000CB
:10370000D83300083F00000049040000E5330008FA
:103710003F00000051040000F33300083F000000A8
:103720000096000000000800040000004835000872
:103730000000000000000000000000000000000089
:08374000000000000000000081
:00000001FF
